:020000040000FA
:1000000004309F009E009C01003065008501FF3098
:1000100066007F30620006080F399D000330061F1E
:100020009D061D080339031903309D040C30861FFB
:100030009D061D080C3903190C309D041D18051070
:100040001D1C05149D1885109D1C85140430061E6A
:1000500005301D1D09309D1D00309F001F081E0228
:10006000031C9E0A1E081F02031C9E0310308506F7
:100070009C099C1C05159C18851556309B00063064
:100080009A009B0B41289A0B41284628472848286C
:1000900049284A280000861A5A28000010309B0080
:1000A00002309A009B0B52289A0B52285728582846
:1000B00059285A28051185111E08861E0A3E8207F6
:1000C0007428822890289D28AA28B828C928D728CB
:1000D000E528F32801290F291D292A293729442930
:1000E0005629632970297E2912309B0004309A001A
:1000F0009B0B78289A0B78287D287E287F288028DB
:1001000000000B2887309B0004309A009B0B862848
:100110009A0B86288B288C288D288E2800000B2887
:100120000D309B0005309A009B0B94289A0B942865
:1001300099289A289B289C280B28A7309B000530DB
:100140009A009B0BA1289A0BA128A628A728A828CB
:10015000A9280B2856309B0006309A009B0BAE282E
:100160009A0BAE28B328B428B528B628B7280B2890
:100170009C309B0006309A000130990001309800B5
:100180009B0BC0289A0BC028990BC028980BC0283D
:100190000B287A309B0007309A009B0BCD289A0BD6
:1001A000CD28D228D328D428D52800000B284B30BE
:1001B0009B0008309A009B0BDB289A0BDB28E02879
:1001C000E128E228E32800000B2836309B000930A4
:1001D0009A009B0BE9289A0BE928EE28EF28F028D3
:1001E000F128F2280B283F309B000A309A009B0B25
:1001F000F7289A0BF728FC28FD28FE28FF2800295D
:100200000B28D0309B0004309A009B0B05299A0BD9
:1002100005290A290B290C290D290E290B283E3006
:100220009B0005309A009B0B13299A0B1329182960
:1002300019291A291B291C290B28E0309B0005309D
:100240009A009B0B21299A0B212926292729282945
:1002500029290B2898309B0006309A009B0B2E29E9
:100260009A0B2E2933293429352936290B286B304E
:100270009B0007309A009B0B3B299A0B3B29402996
:100280004129422943290B28BE309B0007309A00A0
:1002900001309900013098009B0B4C299A0B4C2996
:1002A000990B4C29980B4C2900000B28C9309B0056
:1002B00008309A009B0B5A299A0B5A295F2960290A
:1002C000612962290B28C4309B0009309A009B0BDE
:1002D00067299A0B67296C296D296E296F290B28CC
:1002E000DE309B000A309A009B0B74299A0B74290C
:1002F00079297A297B297C297D290B2819309B00B3
:100300000C309A009B0B82299A0B82298729882915
:0803100089298A298B290B2899
:02400E00F13F80
:1042000041006C0063006F007200200031002E003E
:104210003200200043006F007000790072006900D6
:104220006700680074002000310039003900370051
:1042300020004D002E00200043006F007600690032
:0A4240006E00670074006F006E004E
:00000001FF
